S123C0007EC3237E7FE87EC5E57EC5EF7EC5FA7EC5F67EC6147EC6127EC61B7EC6367EC638
S123C0204A0D0A040D0A3E20040D0A0A4D4333206D6F6E69746F7220312E310D0A44616E38
S123C04069656C20547566766573736F6E20323031330D0A0D0A20472020476F2028525456
S123C06049290D0A204A20204A756D7020746F20616464726573730D0A204C20204C6F6105
S123C080642053312066726F6D20636F6E736F6C650D0A204D43204D656D6F727920636862
S123C0A0616E67650D0A204D44204D656D6F72792064756D700D0A205252205072696E74A2
S123C0C020636F6E74656E7473206F6620737461636B0D0A2052532052657365742073749D
S123C0E061636B20706F696E7465720D0A205243204368616E676520737461636B204343DE
S123C1000D0A205241204368616E676520737461636B20410D0A205242204368616E676523
S123C12020737461636B20420D0A205258204368616E676520737461636B20580D0A2052E5
S123C14050204368616E676520737461636B2050430D0A2050202053656C65637420492F7D
S123C1604F20706167650D0A040D0A43432042202041202058202020205043202020535066
S123C1802020202020482049204E205A205620430D0A040D0A41444452202030202031203B
S123C1A020322020332020342020352020362020372020203820203920204120204220208C
S123C1C0432020442020452020460D0A040D0A4C6F616420533139207265636F72640D0A44
S123C1E0040D0A0A4C6F6164206661696C202D205072657373205920746F20636F6E7469A7
S123C2006E75650D0A040D0A4C6F6164204F4B0D0A040D0A5452415020617420616464724D
S123C2206573733A2024040D0A506172616D65746572206572726F720D0A048E7F00BF7FC5
S123C24008BDC680BDC5A986FF9700868797024F9714CEC024BDC5EFBDC5E5810D27F38432
S123C260DF814826037EC307814726037EC310814A26037EC314815226037EC2C2814D2624
S123C280037EC299814C26037EC4FD815026037EC587863FBD7FE820B9BDC5E5810D2603E5
S123C2A07EC25284DF814326037EC3E2814626037EC424814426037EC472863FBD7FE87E16
S123C2C0C252BDC5E5810D26037EC25284DF815226037EC329814126037EC3738142260342
S123C2E07EC385815826037EC397815026037EC3AF814326037EC3C7815326037EC3D9861E
S123C3003FBD7FE87EC252CEC029BDC5EF7EC252BE7F083B8620BD7FE8BDC64A24036E00BE
S123C3207EC252BF7F087EC252CEC169BDC5EFFE7F0808BDC614BDC614BDC614BDC612BD82
S123C340C612CE7F08BDC6128620BD7FE8FE7F0808E600CE000658588620BD7FE858250807
S123C3608630BD7FE87EC36D8631BD7FE80926E87EC252863DBD7FE8FE7F08BDC636240262
S123C380A7037EC252863DBD7FE8FE7F08BDC6362402A7027EC252863DBD7FE8BDC64A24FF
S123C3A00BFF7F0CFE7F08FC7F0CED047EC252863DBD7FE8BDC64A240BFF7F0CFE7F08FC67
S123C3C07F0CED067EC252863DBD7FE8FE7F08BDC6362402A7017EC2528E7F00BF7F087EF3
S123C3E0C2528620BD7FE8BDC64A242FCEC021BDC5EFCE7F0CBDC612FE7F0CBDC614FF7F8F
S123C4000CBDC636240E09A700A10027DF863FBD7FE820D881DD27D47EC252CEC227BDC5C5
S123C420EF7EC2528620BD7FE8BDC64A2432FF7F0E862DBD7FE8BDC64A2425FF7F0CBC7F4C
S123C4400E231D08FF7F0C8620BD7FE8BDC636240F16FE7F0EE70008BC7F0C26F87EC252BB
S123C460CEC227BDC5EF7EC252CEC227BDC5EF7EC2528620BD7FE8BDC64A24EDFF7F0CCE44
S123C480C021BDC5EFB67F0D84F0B77F0DCEC193BDC5EF8610B77F0BCE7F0CBDC61286204F
S123C4A0BD7FE8FE7F0CFF7F0EBDC614FF7F0CB67F0D840F810826058620BD7FE881002624
S123C4C0E8FE7F0EFF7F0C8620BD7FE8A600817E220481202C02862EBD7FE808FF7F0CB6D7
S123C4E07F0D840F26E6CEC021BDC5EF7A7F0B270220A5BDC5E5810D278B7EC252CEC1CD66
S123C500BDC5EF860DBD7FE88639B77FE8BDC5E5815326F4BDC5E581392757813126E97FDE
S123C5207F0ABDC63616FB7F0AF77F0A8002B77F0BBDC64A2425F67F0AFB7F0CFB7F0DF73F
S123C5407F0ABDC63616FB7F0AF77F0A7A7F0B2705A7000820EC7C7F0A27A8867EB77FE89A
S123C560CEC1E1BDC5EFBD7FEB84DF815926F77EC252BDC5E5810D26F9867EB77FE8CEC2FD
S123C58006BDC5EF7EC252863DBD7FE886FF9700BDC61B240481072309CEC227BDC5EF7E6B
S123C5A0C2528A8097027EC25286059710860A971196123937D61158585824F9971333398A
S123C5C09612961184C0810027F8814027F29612399612961184C081002707814027F286C7
S123C5E00139860039BD7FEB7E7FE8BD7FE808A600810426F63944444444840F8B3081396E
S123C60023028B077E7FE8A600BDC5F6A600087EC5FA8DF38DF186207E7FE8BDC5E58030D1
S123C6202B1281092F0C84DF81112B0881162E0480070D390C39BDC61B240D4848484816EC
S123C640BDC61B24031B0D390C398DEA240DB77F0C8DE32406B77F0DFE7F0C39BF7F08BDDF
S123C660C3297EC252BF7F08CEC212BDC5EFFE7F08C6063ABDC612CEC021BDC5EF7EC2520D
S123C680867ECEC252B77FFDFF7FFECEC65CB77FFAFF7FFBCEC310B77FF7FF7FF8CEC31083
S123C6A0B77FF4FF7FF5CEC310B77FF1FF7FF2CEC310B77FEEFF7FEFCEC5B4B77FE8FF7F8C
S117C6C0E9CEC5C2B77FEBFF7FECCEC5D3B77FE5FF7FE6397B
S105FFEEC665E2
S111FFF27FEE7FF17FF47FF77FFA7FFDC23B45
S9030000FC
